:020000040000FA
:1000000000008A110A12172BF200030E8301F1007F
:100010000A088A01F000040883120313EC0083121B
:1000200003130B1D17288914810189100B118312EA
:1000300003136C08840070088A008301710E83002A
:10004000F20E720E0900DC22831203138B17831643
:100050000313AD010C30831603132D02031840283F
:100060002D08B03EAE0000300318013EAF002E0850
:10007000840083132F188317FF308000AD0A2A28CD
:1000800083160313AD011830831603132D020318D2
:1000900059282D084D3EAE0000300318013EAF0038
:1000A0002E08840083132F18831777308000AD0A41
:1000B0004328932083120313871B5F28F22000300C
:1000C000831203136A0403195A2893205A2808003C
:1000D0000B30831203130102031868280915091055
:1000E00083160313AA010C30831603132A02031884
:1000F0008B282A08B03EAB0000300318013EAC004C
:100100002B08840083132C1883170008D020831633
:100110000313AA0A73288312031309140910831204
:100120000313EB0108000B308312031301020318C1
:100130009328091DA1280911013083160313A1007A
:10014000A42883160313A10183160313A2011830F8
:100150008316031322020318BF2822084D3EA30072
:1001600000300318013EA4002308840083132418E0
:1001700083170008D02083160313A20AA72883122E
:100180000313091409108316031321080319CC283B
:10019000831203138715871183120313EA010800E2
:1001A00083160313A900A601083083160313260241
:1001B0000318F128A91FE028831203138716E328E8
:1001C00083120313871283120313871503108316F8
:1001D0000313A90D83120313871183160313A60AB1
:1001E000D4280800CC2283160313A1002108031988
:1001F00026292108013A03192B292108023A03195B
:1002000030292108033A031952292108803A031999
:10021000B22A2108813A031974292108823A031964
:1002200078292108F03A03197C292108F13A0319A9
:10023000342A2108F23A0319882A2108F53A0319C9
:10024000A42A2108F63A0319AD2AB22A01308312F2
:100250000313EA00B22A013083120313EB00B22A1F
:1002600083160313A1011830831603132102031808
:100270004D2921084D3EA20000300318013EA30085
:10028000CC2283160313A4002208840083132318AE
:10029000831724088000A10A332901308312031335
:1002A000EA00B22A83160313A1010C30831603134C
:1002B000210203186F292108B03EA2000030031864
:1002C000013EA300CC2283160313A400220884005D
:1002D00083132318831724088000A10A55290130AD
:1002E00083120313EB00B22A831203138B13B22A77
:1002F000831203138B17B22A83160313A10105304F
:100300008316031321020318B22A0930FF002108C3
:100310008A110A12DF238A110A1283160313A2001C
:10032000203EA30000300318013EA40023088400EF
:100330008313241883170008A500840A0008A3006B
:100340008403A401A31BA4032308A500B3228316DE
:1003500003132208203EA30000300318013EA4002E
:10036000230884008313241883170008A500840A37
:100370000008A60084032508A300B32283160313F4
:100380002208203EA30000300318013EA5000230E1
:10039000A3070318A50A23088400831325188317CD
:1003A0000008A600840A0008A3008403A501A31B7B
:1003B000A5032308A600B322831603132208203EB8
:1003C000A30000300318013EA5000230A307031864
:1003D000A50A230884008313251883170008A600A4
:1003E000840A0008A70084032608A300B32283160A
:1003F00003132208203EA30000300318013EA6008C
:100400000430A3070318A60A2308840083132618C0
:1004100083170008A700840A0008A3008403A6012C
:10042000A31BA6032308A700B322831603132208E5
:10043000203EA20000300318013EA3000430A207B2
:100440000318A30A220884008313231883170008C3
:10045000A600840A0008A70084032608A200B3228D
:1004600083160313A10A7F2983160313A101053004
:100470008316031321020318B22A0930FF00210852
:100480008A110A12DF238A110A1283160313A200AB
:10049000203EA60000300318013EA7000630A60744
:1004A0000318A70A26088400831327188317000857
:1004B000A800B322831603132208203EA6000030B2
:1004C0000318013EA7000730A6070318A70A26084D
:1004D00084008313271883170008A800B32283160B
:1004E00003132208203EA20000300318013EA6009C
:1004F0000830A2070318A60A2208840083132618CE
:1005000083170008A700B32283160313A10A372A12
:1005100083160313A1011830831603132102031855
:10052000B22A21084D3EA20000300318013EA60069
:10053000220884008313261883170008A700B3221B
:1005400083160313A10A8B2A831203136A08B322AA
:10055000831203136B08B322B22ACC22831603132F
:10056000A100B322080083160313A0008312031313
:10057000071BB62A8316031388018312031306147C
:100580008316031320088312031388000610FF301C
:10059000831603138800080083120313871BCC2AD9
:1005A0008610080883160313A00083120313861411
:1005B0008316031320080800831203138B018101A3
:1005C0008B1697019D019401831603138C018D01F5
:1005D00083120317870188017830831603138F0075
:1005E000033081008312031385018601870188018E
:1005F00089018614061489140910871183160317BC
:100600008801831603138501831603178901C830F7
:10061000831603138600D0308700FF3088008901DD
:1006200083120313EA0183120313EB010800FC3069
:10063000FE000330FF0080308A110A12BE238A11A7
:100640000A1283160313BD007F08BC00FE30BE00F3
:100650000330BF00831603133C08C0003D08C100EF
:10066000FF30BC07031CBD03400841040319A72B3E
:1006700004303E07C000C101C10D3F08C10740085A
:10068000FE004108FF0080308A110A12BE238A1141
:100690000A1283160313C3007F08C2003E08FE003F
:1006A0003F08FF0080308A110A12BE238A110A1205
:1006B00083160313C500C1007F08C400C0000230C8
:1006C0003E07C000C101C10D3F08C1074008FE0040
:1006D0004108FF0080308A110A12BE238A110A12D3
:1006E00083160313C100C7007F08C000C60083162D
:1006F00003134208C6004308C700FF30C207031CAB
:10070000C303460847040319A02B4408FE0045080C
:10071000FF0080308A110A12AB238A110A12831655
:100720000313C6004008840083134118831746084A
:100730008000C40A0319C50AC00A0319C10A772B2D
:10074000063083160313BE070318BF0A2A2B8A112B
:100750000A1223280800003A0319B22B803A031921
:10076000B92B00347E08840083137F188317000898
:1007700008007F088A007E0882000800003A0319FA
:10078000C62B803A0319D02BFF0100347E08840069
:1007900083137F1883170008FF00840A00080800ED
:1007A0008A110A12B923FD00FE0FFF03FF0A8A1106
:1007B0000A12B923FC007D08FF007C0808008312A0
:1007C0000313E5007F08E600E7010830E800831224
:1007D0000313651CED2B6608E707831203136508F6
:1007E000E9000310690CE5000310660DE900E6005E
:1007F000E80BE72B670808000134003404340434A4
:0A0800006D3400340134003400347C
:02400E00F5209B
:02401000FC3F73
:00000001FF
